:100000000C9482040C94B2040C94B2040C94B204C8
:100010000C94B2040C94B2040C94B2040C94B20488
:100020000C94B2040C94B2040C94B2040C94B20478
:100030000C94B2040C94B2040C94B2040C94B20468
:100040000C94B2040C94B2040C94B2040C94B20458
:100050000C94B2040C94670A0C94B2040C94B2048D
:100060000C94B2040C94B2040C94B2040C94B20438
:100070000C94B2040C94B2040C94B2040C94B20428
:100080000C94B2040C94B2040C94B2040C94B20418
:100090000C94B2040C94B2040C94B2040C94B20408
:1000A0000C94B2040C94B2040C94B2040C94B204F8
:1000B0000C94B2040C94B2040C94B2040C94B204E8
:1000C0000C94B2040C94B2040C94B2040C94B204D8
:1000D0000C94B2040C94B2040C94B2040C94B204C8
:1000E0000C94B2040C942A0502FDFFC80002FCFF28
:1000F000C80002FBFFC80002FDFFC80002FCFFC8E9
:100100000002FBFFC80002FDFFC80002FCFFC800A0
:1001100002FBFFC80002FDFFC80002FCFFC800028E
:10012000FBFFC80002FDFFC80002FCFFC80002FB85
:10013000FFC80002FDFFC80002FCFFC80002FBFF71
:10014000C80002FDFFC80002FCFFC80002FBFFC898
:100150000002FDFFC80002FCFFC80002FBFFC80050
:1001600002FDFF900102FCFF900102FBFF900102E3
:10017000FDFFF40102FCFF260202FBFF580202FD14
:10018000FF200302FCFF840302FBFFE803000000E2
:10019000E803000000000002FEFF500002FDFF50D7
:1001A0000003FCFFAA000000001E0003FAFFAA00E3
:1001B0000000001E0003FAFFAA000000001E00025B
:1001C000FEFF500002FDFF500003FCFFAA000000EC
:1001D000001E0003FAFFAA000000001E0003FAFF41
:1001E000AA000000001E0002FEFF500002FDFF50AA
:1001F0000003FCFFAA000000001E0003FAFFAA0093
:100200000000001E0003FAFF2C0103FCFF82000324
:10021000FEFF8200000000500002FFFF500002FEBF
:10022000FF500003FDFFAA00000000140003FBFFC5
:10023000AA00000000140003FBFFAA000000001E3B
:100240000002FFFF500002FEFF500003FDFFAA0066
:10025000000000140003FBFFAA00000000140003CC
:10026000FBFFAA00000000140002FFFF500002FE86
:10027000FF500003FDFFAA000000001E0003FBFF6B
:10028000AA000000001E0003FBFF2C0103FDFF82FB
:100290000003FFFF8200000000500000000000008B
:1002A0000200006400020A00640002000064000210
:1002B0000A0064000200006400040000C800010A93
:1002C00000320001F6FF3200010A00320001F6FFA1
:1002D00032000200006400020A00640002000064B0
:1002E00000020A0064000200006400040000C8006C
:1002F000010A00320001F6FF3200010A003200015B
:10030000F6FF32000200006400020A0064000200EE
:10031000006400020A00640002000064000400009F
:10032000C800010A00320001F6FF3200010A003263
:100330000001F6FF32000200006400020A006400BF
:100340000200006400020A0064000200006400046D
:100350000000C800010A00320001F6FF3200010A65
:1003600000320001F6FF32000200006400020A00C1
:1003700064000200006400020A00640002000064DD
:1003800000040000C800010A00320001F6FF32003C
:10039000010A00320001F6FF320002FEFF64000293
:1003A0000800640002FEFF6400020800640002FE10
:1003B000FF6400040000C800010C00320001F8FFD7
:1003C0003200010C00320001F8FF320002FDFF6430
:1003D00000020700640002FDFF64000207006400E1
:1003E00002FDFF6400040000C800010D003200019E
:1003F000F9FF3200010D00320001F9FF3200000068
:10040000000000300C03DF31FA2B78D5D86C294579
:10041000A1026969918D6571B843DEF2F6786E1DAF
:10042000BF344ECB382EFD3259750732E231778416
:1004300033E1EDC56E5236279615198D8D88AB4D7B
:10044000BCF918F5271627818C2FB46E602BF29417
:100450000CE0597B338FA3C9A4BD573245027F02FC
:10046000FB98F723AE1EA53A4D59A9AE849B429145
:100470007C9B0CB02BB07ACF6DD102B2D381B4CEBD
:1004800019ACF2C7CB970218F0ABC774470906C482
:10049000A51374D0C3EEA030BFA2E2922497613DB1
:1004A0004453050FEA0728DAB3EF4FFAF955BE9F18
:1004B00068336F2B21105CE0B23F73D6D7D4141B86
:1004C000271A2A122153ECD5423CCF3C918EDBFAFD
:1004D000C24B26E35B82C40EC137E5980BFAB433F6
:1004E00014DE453631320B746EDBB1006A8CFA2CA7
:1004F000D7210F33A3D342650A27FE1621B249350F
:10050000918E6BC3C077382E52E92FBC7629E84D07
:100510004BF781EFCBC354D5EB53EC0D0635439825
:10052000C3AF5B842694B3787DE235F30C1D41574D
:1005300015C346E0879BB672EEA37FF5D8C28D9CAB
:1005400072E920987DD311FBB546EFC1643119796A
:10055000F45F5A7BFA11EEE9B46EDE8C316C29A39C
:1005600055493BD31C4DCED293BE94F7EFAD71E409
:100570000DCC6008DD4EF192BCD01FED3C4890924E
:1005800091CC65AE193481ADF215A5E2C317C6D082
:10059000E327D8C175CA53329B721FD8BBB06A4DCE
:1005A0007DD0FB97047D45F793EAD95601A027E457
:1005B000C700A53DCBF96F666C8F3F2740A974BE7D
:1005C0007A70557FEE9A76818550D787F1FF6BB9A7
:1005D000FF11F7CA0B673177F7709F371A14F6943B
:1005E000854B1373E68AF46CDBCBF3CCCB5F86CA06
:1005F000717D957CE4C6F4DC36931350A70AE52D93
:1006000055F9A03C8394A95F609C2B2BFCB2F66D3E
:10061000308BE91451DEF0887104D8190EBE46649F
:10062000B7E6A13B7B4A9ADBE7C607E378FD51A812
:10063000883BBDDA19AE628AB33AA4C2F9EB26B0A0
:10064000D2C8EC4D138629FA4D30DEC62E2F6FB678
:100650006A2D9083DBF20E8F2DB351279E78D871CF
:1006600040C4BE544BE84E98182D5F465DCEFDC782
:10067000FB8E4BD7815A66AF0EB7D6AC2FAE1D702E
:1006800072DCC4BDC41356DD40B6249D8421658050
:10069000B0B157310BBDE01975B6C6A564E415D7E6
:1006A000C1DA9585EDEC632EA287CC26A932A65936
:1006B000E3FD8AEFBB6B093021CFD586B4EB5D75C6
:1006C000C5F3FBB3DF5EE281E6AFA78FE14EE8C57D
:1006D0004C73B407DFBE38018E0D8742F8E5B8BE13
:1006E000D8B472B7125439F904E088E62F71AB7BA5
:1006F000E56083C41EBBC5ACC94DEFC233A7800CF7
:100700005BF3C36E48FC674CDDF0320D61DD88475A
:100710003E0B0B5CC7D109901EF852529FD25EFB74
:10072000C622690E1FD15AFDC28C0A236A926AA999
:100730009E760565470EF5660647B9A61A17A2E02C
:10074000390CEE59DD49569FD660C341F32EEA912C
:10075000A4F0F7ECFEEC5305340CAC4F244E2F5DA7
:100760005A1EB738670DD83E6D9C7F61CA69F26F1B
:1007700059E95C58D6B05E0BBC0A5AE0598A3EB4BF
:10078000A8F5EC1003C54E7161CED22C37C49C91F4
:10079000AEF8EA85A848906552EB46AC7584601EB9
:1007A0007A4D2F7D137DEE744CC0A183853D1534A9
:1007B00036FFBADF474B449A368A47AC0FA7CA893F
:1007C000F5F9070877F57DC3B61F473C5C5C71936C
:1007D0005C2B72A376B73EAC418558512D23DB22AA
:1007E0001CE22B93D8A8578FC79ECB24FB3CB7574E
:1007F000682AFBDEE1398B23BFE474EC074F0F243A
:10080000323AB87F8285888C8F9295989B9EA1A45E
:10081000A7AAADB0B3B6B9BBBEC1C3C6C9CBCED013
:10082000D3D5D7D9DCDEE0E2E4E6E8E9EBEDEEF0A3
:10083000F1F2F4F5F6F7F8F9FAFBFCFCFDFDFEFE2B
:10084000FEFEFEFEFEFEFEFEFDFDFCFCFBFAFAF9DE
:10085000F8F7F6F4F3F2F0EFEDECEAE8E7E5E3E1C0
:10086000DFDDDBD8D6D4D1CFCCCAC7C5C2BFBDBAB5
:10087000B7B4B1AFACA9A6A3A09D9A9693908D8A68
:100880008784817D7A7774716E6B6864615E5B5872
:1008900055524F4D4A4744413F3C393734322F2D52
:1008A0002A282623211F1D1B1917161412110F0E9B
:1008B0000C0B0A08070605040403020201010000EC
:1008C0000000000000000000010102020304050610
:1008D0000708090A0C0D0E1011131516181A1C1E04
:1008E00020222527292B2E303335383B3D404345E8
:1008F000484B4E5154575A5D606366696C6F72760F
:10090000797C7F0011241FBECFEFD1E2DEBFCDBFC7
:1009100000E00CBF84B78093E80D14BE0FB6F894C6
:10092000A8958091600088618093600010926000BB
:100930000FBE1DE0A0E0B2E0E4EAFCE100E00BBF86
:1009400002C007900D92A235B107D9F72DE0A2E5BC
:10095000BDE001C01D92A83EB207E1F70E942D0B39
:100960000C94500E0C940000CF93C62F0E948F0A57
:100970008FEF80BBC1BBEBE0F1E08081857F80839E
:1009800085E08A95F1F7000080818A608083CF91AD
:1009900008950E948F0A10BA11BAEBE0F1E080814D
:1009A000837F808385E08A95F1F700008FB1908185
:1009B0009C609083089563E883E00E94B40463E040
:1009C00080E00E94B40460E081E00E94B40463E02F
:1009D00083E00E94B40480E092E09093E50D809360
:1009E000E40D87EC92E00C94850BCF93DF93CDB7A9
:1009F000DEB7FE01369681919191BF010E94B10B45
:100A00008AE090E00E947F0B90E080E0DF91CF9140
:100A10000895CF92DF92EF92FF92CF93C82F80E498
:100A2000C82E82E4D82E8FE0E82EF12C85E00E94BB
:100A3000C90485FD06C081E0C81AD108E108F108A3
:100A4000A9F76C2F80E0CF91FF90EF90DF90CF90CF
:100A50000C94B404CF93C82F8091520D8F5F809374
:100A6000520DC03259F4873480F070E060E08AE0C3
:100A70000E942A0590E080E0CF910895CA3029F4C1
:100A80001092520D8DE00E9409058C2F0E940905DD
:100A9000F1CFCF9385E00E94C90480FF0FC080E0B2
:100AA0000E94C904C82F0E94C906CD3019F48AE0FB
:100AB0000E9409058C2FCF910C940905CF910895C0
:100AC000CF93C62F0E948F0A8FEF80BBC1BBEBE094
:100AD000F1E080818D7E808385E08A95F1F70000CA
:100AE000808180618083808182608083CF9108953E
:100AF0000E948F0A10BA11BAEBE0F1E080818B7E80
:100B0000808385E08A95F1F700008FB19081946130
:100B1000908308950F931F93CF93DF9380910F02DB
:100B2000833009F4B3C0A8F4813009F444C0CFE79E
:100B3000823009F476C0C0E060E08C2F81700E94A2
:100B40006005CF5FCF3FC1F7DF91CF911F910F912C
:100B50000895843009F4C8C01FE7CFEFD0E00FEF4D
:100B6000853049F76091590D8FEF860F8E3F28F041
:100B700080910E02819580930E0280E00E946005B4
:100B80006091590D81E00E9460054091530D509194
:100B9000540D57FDDFC08091570D9091580D01966F
:100BA000841795070CF0CAC09093580D8093570D89
:100BB0001150C1F6C9CFCFE7E091590DF0E0ED5FDC
:100BC000F74F649181E00E946005E091590DF0E0DB
:100BD000ED5FF74F649180E00E9460052091530D16
:100BE0003091540D37FD19C08091570D9091580DDB
:100BF0000196821793073CF49093580D8093570DFC
:100C0000C150D1F6A1CF1092580D1092570D80917E
:100C1000590D8F5F8093590DF3CF8091590D821B31
:100C2000F9CF8091590D87FF1DC06FEF80E00E94C2
:100C300060056FEF81E00E9460052091530D3091B7
:100C4000540D37FD1FC08091570D9091580D01969E
:100C5000821793076CF49093580D8093570DC150F1
:100C600001F772CF60E080E00E94600560E0E2CFB3
:100C70001092580D1092570D8091590D8F5F8093EF
:100C8000590DEDCF8091590D821BF9CFCFE76091BF
:100C9000590D80E00E9460056091590D81E00E942D
:100CA00060052091530D3091540D37FD19C080918E
:100CB000570D9091580D0196821793073CF490932D
:100CC000580D8093570DC15011F73ECF1092580D1B
:100CD0001092570D8091590D8F5F8093590DF3CF6E
:100CE0008091590D821BF9CFCFE7E091550DF0911E
:100CF000560DED5FFB4F649181E00E946005E0912D
:100D0000550DF091560DED5FFB4F649180E00E9410
:100D100060058091550D9091560D0196811524E046
:100D2000920738F49093560D8093550DC150E9F613
:100D30000BCF1092560D1092550DF8CF1092580D02
:100D40001092570D8091590D90910E02890F80934A
:100D5000590D2ECF20910E022403B001259F700D56
:100D600011248091590DFE01E81BF109E617F707E0
:100D70001CF40093590D1CCF249F202D1124209387
:100D8000590D16CF80E00E94780580FF0C948A05EB
:100D9000089590915C0DE92FF0E0E359F24F8F3701
:100DA00029F4915090935C0D108208959F5F909369
:100DB0005C0D80830895FF920F931F93CF93DF9371
:100DC000F62EC82FD0E08E01000F111FF801E75852
:100DD000FD4F81818F9380818F930E94F504CF52C4
:100DE000D24F0F900F908881882311F0F11012C01C
:100DF00081E0888370E060E08AE00E942A05F801C3
:100E0000EB59FD4F81818F9380818F930E94F50470
:100E10000F900F90DF91CF911F910F91FF90089548
:100E2000CF93DF93C82FD0E0E091100284E0E89FD9
:100E3000F0011124E35CFD4FEC0FFD1F8081811157
:100E40000DC08091AA028F938091A9028F930E9476
:100E5000F5040F900F90DF91CF910895FE01EE0FF2
:100E6000FF1FE157FD4F81818F9380818F938DEC20
:100E700092E09F938F930E94F504E091100284E02A
:100E8000E89FF0011124E35CFD4FEC0FFD1F808112
:100E90008093100261E00E94DB06E0911002F0E016
:100EA000EE0FFF1FEF5EFD4F808191819093610DEA
:100EB0008093600D0F900F900F900F90CCCFEF921A
:100EC000FF920F931F93CF93DF930BED1DE0F8017B
:100ED000819181110DC08DE0E23EF807C9F780EFE6
:100EE00092E09F938F930E94F5040F900F9028C07B
:100EF00086EE92E09F938F930E94F5040F900F90DF
:100F0000D0E0C0E08FEDE82E82E0F82EF80181916C
:100F10008F01882389F0FE01EE0FFF1FE15DFD4F79
:100F200081818F9380818F93FF92EF920E94F504CD
:100F30000F900F900F900F902196C730D10531F789
:100F4000DF91CF911F910F91FF90EF900895E09165
:100F50001002F0E0EB5DFD4FE081E7FF0BC08091F8
:100F6000AE028F938091AD028F930E94F5040F9093
:100F70000F900895EE0FFF0BE15DFD4F81818F9380
:100F800080818F9388E093E09F938F930E94F50474
:100F90000F900F900F900F900895CF92DF92EF92E5
:100FA000FF920F931F93CF93DF93D82FF92EE091E9
:100FB0001002F0E0EB5DFD4FC0800FE212E0C0E0F8
:100FC000C7FE0BC08091AE028F938091AD028F93CC
:100FD0000E94F5040F900F9034C0F801E080D1809A
:100FE0000E5F1F4FAE2DBD2DFD0101900020E9F7D2
:100FF0003197AF014A1B5B0B6D2F7F2D8E2D9D2DE1
:101000000E94670B892B31F5CC1228C0DF92EF923A
:1010100087E193E09F938F930E94F504E091100283
:10102000F0E0EB5DFD4FA0810A2E000CBB0BA5523A
:10103000B24F81E08C938FEF80830F900F900F90D1
:101040000F90DF91CF911F910F91FF90EF90DF9064
:10105000CF900895CF5FC73009F0BFCF87E293E00C
:101060009F93B5CF97E0EBEDFDE0DF01292F1D92B7
:101070002A95E9F7E1EDFDE0DF011D929A95E9F788
:10108000E5E2F2E09FEF9193B2E0EF32FB07D9F790
:10109000882319F11092100281E08093E10D85E020
:1010A0008093290281E080932A0282E080932C02BF
:1010B00010925B0D10924D0280911002E82FF0E02B
:1010C000EE0FFF1FEF5EFD4F208131813093610DE8
:1010D0002093600D60E00C94DB0680915A0D88230C
:1010E00079F081E0809310028091C5029091C60250
:1010F00090936A028093690284E080932702CFCFA5
:1011000081E0809310021092450283E080932702D1
:1011100086E08093260210922D02C1CFCF938230B9
:10112000A1F480915B0D811145C081E080935B0D3E
:101130001092DD0D8AE393E09F938F930E94F50454
:101140000F900F9081E0CF91089581110CC0809194
:101150005B0D813079F582E080935B0D1092DB0DA1
:1011600085E593E0E9CF843091F4C0915B0DC13007
:1011700009F582E080935B0D1092DF0D81E793E02B
:101180009F938F930E94F504C0935D0DD9CF81305A
:1011900089F480915B0D823069F41092DC0D8EE948
:1011A00093E09F938F930E94F50480915D0D0E94C0
:1011B0003208C6CF80E0C7CFE82FF0E0E552F24F0B
:1011C0009081911106C08091A6028F938091A50213
:1011D00037C0853009F443C078F4833021F184307E
:1011E00011F0833081F390911002993061F70E94E1
:1011F0008E08882341F30895863029F780911002E4
:10120000823011F583E0809345028091B0028F9384
:101210008091AF028F930E94F50481E080935A0D74
:101220000F900F90E8CF90911002923061F61092DB
:10123000DE0D809345028091B6028F938091B502B6
:101240008F930E94F504ECCF8111BDCF8CEF93E01A
:101250009F938F930E94F5041092E10DE1CF90913E
:101260001002943009F0AFCF1092E00D80934D0240
:101270008091BC028F938091BB02E2CFEF92FF92EC
:101280000F931F93CF93DF93182F092F8FE2E82E30
:1012900082E0F82ED0E0C0E0F701819191917F01CA
:1012A000FC0101900020E9F73197AF01481B590B71
:1012B000612F702F0E94670B892B49F48C2FDF91CF
:1012C000CF911F910F91FF90EF900C94DC08219625
:1012D000C730D10509F78091A6028F938091A502AE
:1012E0008F930E94F5040F900F90DF91CF911F9183
:1012F0000F91FF90EF9008950F931F93CF93DF937B
:10130000C82F70E060E08AE00E942A05C73009F427
:1013100055C0B8F5C53009F448C0C63009F454C00A
:101320008FEF8C0F843008F446C080E694E09F93E2
:101330008F930E94F504CDE8D2E00F900F900FED4F
:1013400012E08881998122969F938F931F930F9328
:101350000E94F5040F900F900F900F9082E0C13A19
:10136000D80779F78091A8028F938091A7028F9375
:101370000E94F5040F900F90DF91CF911F910F9174
:101380000895C830F1F0C93081F6E0919F02F091E4
:10139000A002DF010D900020E9F7CD018E1B9F0B0D
:1013A0008359924F0E94CD07DDCF60E080911002FB
:1013B0000E94DB06D7CF0E941007D4CF0E945F07A0
:1013C000D1CF0E94A707CECFE0919902F0919A0267
:1013D000DF010D900020E9F7CD018E1B9F0B835993
:1013E000924F0E943E09BECF0F931F93CF93DF937E
:1013F000E0915C0DE436B0F010925C0DEDE6FDE09E
:1014000084E6DF011D928A95E9F789E694E09F93CF
:101410008F930E94F5040F900F90DF91CF911F9151
:101420000F910895F0E0E459F24F80818A3011F075
:101430008D3099F70DE812E0D0E0C0E0F80181911D
:1014400091918F01FC0101900020E9F73197AF01E4
:10145000481B590B6DE67DE00E94670B892B69F4F0
:101460008C2F0E947C0910925C0DEDE6FDE084E675
:10147000DF011D928A95E9F7D0CF2196CA30D105B8
:10148000E9F68091A4028F938091A3028F930E942A
:10149000F5040F900F90E7CF8091C3029091C402A2
:1014A00090936A02809369028091BD029091BE027E
:1014B0009093A8028093A702089582E884BD84E0F7
:1014C00085BD80E487BD82E080936E0008951F9201
:1014D0000F920FB60F9211240BB60F922F933F93DA
:1014E0004F935F936F937F938F939F93AF93BF932C
:1014F000EF93FF930E94B40AFF91EF91BF91AF91D8
:101500009F918F917F916F915F914F913F912F911B
:101510000F900BBE0F900FBE0F901F9018958093E9
:10152000080108958FEF80BB8093070180930A0123
:101530001092080111BAEBE0F1E0108280818F6116
:1015400080838FE891E00197F1F700C0000080816F
:101550008E7F808308950E94C2060E9449050E94E2
:10156000F40990E080E008956091600D7091610D44
:101570006115710529F410926C0D10926B0D089590
:1015800080916B0D90916C0D019690936C0D8093F2
:101590006B0D2091640D3091650D4091690D509156
:1015A0006A0D8417950720F46217730721F40895D4
:1015B0006217730761F01092630D1092620D109222
:1015C0006C0D10926B0D7093650D6093640D2091FE
:1015D000620D3091630D45E0429FC001439F900D25
:1015E0001124680F791F45E050E086E69DE00E94D7
:1015F0005E0B8091690D90916A0D892B71F41092A8
:10160000630D1092620D6091600D7091610D45E067
:1016100050E086E69DE00E945E0B8091660D80930F
:101620000F028091670D9091680D20915E0D3091B1
:101630005F0D820F931F9093540D8093530D109262
:101640006C0D10926B0D8091620D9091630D01965F
:101650009093630D8093620D0895F8940E94920A0E
:101660000E94DB040E945D0A0E944C0A88EE90E012
:101670009093610D8093600DE1EDFDE08AE0DF0164
:101680001D928A95E9F7EBEDFDE087E0DF011D9201
:101690008A95E9F760E0809110020E94DB06789459
:1016A00088E199E20FB6F894A895809360000FBE88
:1016B00090936000A8950E94AB0AFCCFFB01DC016F
:1016C00002C005900D9241505040D8F70895FB019B
:1016D000DC014150504088F08D9181341CF08B35F5
:1016E0000CF4805E619161341CF06B350CF4605E2B
:1016F000861B611171F3990B0895881BFCCF6091D3
:10170000E40D7091E50D0C94C20D0F931F93CF93D0
:10171000DF93E091E40DF091E50D238110E000E00E
:1017200021FD0EC00FEF1FEFC801DF91CF911F9178
:101730000F9108951995892B11F00FEF1FEFCE012E
:10174000EC0189916091E40D7091E50DDB01189633
:10175000ED91FC918111EECF8AE01995892B21F34F
:10176000E1CFAB01BC018091E40D9091E50D0C94AB
:10177000B90B2F923F924F925F926F927F928F920E
:101780009F92AF92BF92CF92DF92EF92FF920F9310
:101790001F93CF93DF9300D000D000D00F920F9211
:1017A000CDB7DEB77C013B018A01FC0117821682AE
:1017B000838181FFCEC19AE0292ECE0101965C0182
:1017C000F7019381F30193FD859193FF81913F018F
:1017D000882309F446C1853239F493FD859193FF3E
:1017E00081913F01853229F4B70190E00E94C20D3A
:1017F000E7CF912C412C512CFFE1F51538F08B32BD
:1018000009F188F4803201F1833221F157FC3AC0AA
:1018100020ED280F2A3040F556FE1FC0929C200D67
:101820001124922E06C08D3291F0803379F768949E
:1018300050F8F30193FD859193FF81913F01811150
:10184000DBCF20C0689451F8689452F8F2CF6894C6
:1018500053F8EFCF689454F8ECCF429C200D11243C
:10186000422E689455F8E5CF8E3229F456FCF9C023
:10187000689456F8DECF8C3619F4689457F8D9CFAF
:101880008836B9F2982F9F7D95549330C0F08336F7
:10189000A1F18337C1F1833509F05BC0F801C19034
:1018A000D1908F01692D70E056FC02C06FEF7FEF81
:1018B000C6010E94AC0D4C01689457F80AC00C5F39
:1018C0001F4F2FE3298388248394912C6501E8948A
:1018D00057F853FC04C04814190409F018F5342CC7
:1018E0008114910431F5332009F46ACFB70180E205
:1018F00090E00E94C20D3A94F6CFF801808189836E
:101900000E5F1F4FE0CFF801C190D1908F01692D7C
:1019100070E056FC02C06FEF7FEFC6010E94B70D6A
:101920004C01D5CFB70180E290E00E94C20D4A94ED
:10193000D2CFF60157FC859157FE81916F01B70117
:1019400090E00E94C20D31103A94F1E08F1A910894
:10195000C7CF843619F0893609F074C0F80157FEF4
:101960006AC061917191819191918F01252D2F769E
:10197000D22E97FF09C090958095709561957F4F05
:101980008F4F9F4F6894D7F82AE030E0A5010E945E
:10199000F20DC82ECA188C2C5D2CD6FE0CC0E89413
:1019A00050F8C91440F4D4FE05C0D2FC03C0FD2D8C
:1019B000FE7E5F2E892C54FEA4C0FE01EC0DF11DAD
:1019C0008081803309F096C0252D297E522E852DE9
:1019D0008870382E53FCA4C050FE9EC09C2C8414EA
:1019E00018F44C0C942C981854FEA0C0B70180E356
:1019F00090E00E94C20D52FE09C088E790E051FEBF
:101A000002C088E590E0B7010E94C20DC91408F435
:101A100099C0CA94D12C9FEFC91AD90ACA0CDB1CF1
:101A2000F60182916F01B70190E00E94C20DAC14E3
:101A3000BD04B1F758CF61917191072E000C880B4E
:101A4000990B93CFD52CE894D4F82AE030E0853771
:101A5000E1F1952D997FD92E8F36A9F1F0F48835D3
:101A600051F1F701868197812B960FB6F894DEBF6E
:101A70000FBECDBFDF91CF911F910F91FF90EF90DF
:101A8000DF90CF90BF90AF909F908F907F906F909E
:101A90005F904F903F902F900895803749F088379E
:101AA00001F7D4FE02C06894D2F820E130E00DC006
:101AB0006894D4F8F6CF54FE03C0E92FE660DE2E1A
:101AC00020E132E002C028E030E0F801D7FE0DC08E
:101AD00061917191819191918F01A5010E94F20D07
:101AE000C82ECA18E894D7F856CF6191719190E04A
:101AF00080E0F2CF52FC02C0839469CF8394839438
:101B000066CF852D867809F462CFF6CFB70180E2E3
:101B100090E00E94C20D83948414C0F3312C64CFF2
:101B2000342C3818841408F45FCFF8CF852D8678CC
:101B300009F46CCF8BE251FE80E257FC8DE2B701D5
:101B400090E062CFB70180E390E00E94C20D9A94CA
:101B50005DCF8FEF9FEF88CFFC0105906150704003
:101B60000110D8F7809590958E0F9F1F0895FC0166
:101B70006150704001900110D8F7809590958E0FBC
:101B80009F1F08950F931F93CF93DF93182F092F53
:101B9000EB018B8181FD09C01FEF0FEF812F902F8B
:101BA000DF91CF911F910F91089582FF14C02E8174
:101BB0003F818C819D81281739073CF4E881F981A8
:101BC000CF0101969983888310838E819F8101962E
:101BD0009F838E83E3CFE885F985812F1995892B23
:101BE000A1F3DACFFA01AA27283051F1203181F18F
:101BF000E8946F936E7F6E5F7F4F8F4F9F4FAF4F15
:101C0000B1E03ED0B4E03CD0670F781F891F9A1F27
:101C1000A11D680F791F8A1F911DA11D6A0F711DDB
:101C2000811D911DA11D20D009F468943F912AE0E7
:101C3000269F11243019305D3193DEF6CF010895CF
:101C4000462F4770405D4193B3E00FD0C9F7F6CF00
:101C5000462F4F70405D4A3318F0495D31FD4052C8
:101C6000419302D0A9F7EACFB4E0A695979587955E
:101C700077956795BA95C9F700976105710508953D
:101C80009B01AC010A2E06945795479537952795E9
:101C9000BA95C9F7620F731F841F951FA01D089581
:041CA000F894FFCFE6
:101CA40000000002000000002A05000000000101FD
:101CB40001E8009701A0029701A0020000000000C3
:101CC4000000000000FF0603FF0501FF0200FF7A89
:101CD40004860492049B04A304A904AD0400000038
:101CE40000020000000001000000020400000000E7
:101CF40003070409060800050000050000000600AB
:101D04000000000005B40448050000D10580062940
:101D140007C707660810096409460A4E0A5A0A6882
:101D24000A720A7D0A870A930A990AA20AB00AB5B6
:101D34000ABB0AC10AC60ACB0AD40AD80AE20AE9CB
:101D44000AEE0AF40A050B0000190B300B410B597B
:101D54000B610B6D0B830B920BA10BB00BC60B002D
:101D6400000000E00B970C494E49540D004D6F766E
:101D7400696E6720746F7761726473202573002025
:101D8400202020257300596F7520686176653A001C
:101D9400596F757220696E76656E746F72792069F9
:101DA4007320656D70747900596F7520666F756E58
:101DB40064206120257300596F7520746F6F6B2048
:101DC40074686520257300546861742773206E6FEE
:101DD4007420686572652E2E2E00596F7520636F0E
:101DE4006E6E656374656420746865206B657962E2
:101DF4006F61726400596F7520696E7365746564F0
:101E04002074686520666C6F707079206469736BE8
:101E140000596F7520696E73657274656420746807
:101E24006520666C65736820696E746F20746865DC
:101E340020666C6F70707920647269766500596FE2
:101E4400752073746172742074686520636F6D709B
:101E5400757465722077697468207468652073638B
:101E64007265776472697665722C20736974206474
:101E74006F776E20616E6420776174636820697483
:101E840020626F6F7420696E746F206120746578AE
:101E940074616476656E747572653A00596F752065
:101EA40063727920666F722068656C702E204974A5
:101EB4002773206E6F207573652E20596F7520610E
:101EC4007474656D707420746F2073686F6F742000
:101ED400796F757273656C662E2049742773206E52
:101EE4006F207573652E2E2E20596F752072756EB6
:101EF400206F7574206F662062756C6C6574730056
:101F0400596F752063616E3A000A546F6F206D75C6
:101F1400636820696E7075742100464C4F505059A7
:101F2400204449534B005343524557445249564564
:101F340052004B4559424F4152440053415553417D
:101F4400474500464C455348004B455900504953BA
:101F5400544F4C00596F7520737461726520696E1B
:101F6400746F206120766F6964206F66206E6F74D1
:101F740068696E676E6573732E20596F752073657B
:101F840065206E6F6F6E652C20796F7520686561B2
:101F940072206E6F6F6E652C796F75206665656C47
:101FA40020736F6D656F6E652E20596F75206C6F91
:101FB4006F6B2061726F756E642C20616E64207388
:101FC4006565206E6F7468696E672C20796574206E
:101FD400796F7520617265206E6F206C6573732054
:101FE4007363617265642E00596F75206172652098
:101FF4006F6E20746865206465616420656E64207A
:102004006F662061206C6F6E656C7920726F6164FD
:102014002E20596F75206C6F6F6B2072696768741E
:1020240020616E64206C656674206F6620796F751C
:102034002C2062757420796F752063616E6E6F74E5
:102044002072656D656D6265722077687920796F9D
:10205400752061726520686572652E2E2E20596F79
:102064007520617265207465727269666965642E93
:1020740000596F752066696E642061206669726517
:10208400706C61636520696E20746865206D696495
:10209400646C65206F662074686520776F6F647365
:1020A4002E204120737472656574206C65616473BD
:1020B40020746F2069742066726F6D2074686520C7
:1020C400776573742E20546865206669726520698B
:1020D4006E20746865206D6964646C65206F662089
:1020E40074686520706C616365206973207374691A
:1020F4006C6C206275726E696E672061732069660C
:1021040020736F6D656F6E6520686164206C656611
:102114007420696E20612068757272792E2E2E00EB
:10212400596F752074726176656C20646F776E20C8
:1021340074686520726F61642E204974206861732D
:10214400206E6F206C69676874732C20627574202C
:10215400746865206D6F6F6E207368696E65732097
:102164006272696768742E2054686520726F6164B6
:1021740020656E64732077697468206120686F75C8
:10218400736520746F20796F7572206C6566742E88
:102194002054686520686F7573657320646F6F726F
:1021A400206D617420697320696E207468652072E3
:1021B4006F61642E2049747320646F6F7220697399
:1021C400206C6F636B65642E00596F7520656E74A7
:1021D400657220746865206C6F6E672068616C6C32
:1021E400776179206F6620746865206F6C6420685D
:1021F4006F7573652E2049742068617320646F6F56
:102204007273206F6E20616C6C2077616C6C732E1E
:102214002054686520646F6F7273206C6F6F6B203D
:1022240061206C6974746C652077656972656420DB
:102234006265636175736520746865792061726590
:1022440020666C617420616E6420646F6E27742054
:102254006861766520612068616E646C6520746FC6
:102264002070756C6C2E00596F7520656E746572E4
:102274002061206C6172676520726F6F6D207769D1
:1022840074682061206665772063686169727320D1
:10229400616E642061207475626520545620696EF5
:1022A400736964652069742E20496E207468652002
:1022B40063656E7465722074686572652069732045
:1022C400612074696C65207461626C65207769743F
:1022D400682061207661736520616E6420666C6F8E
:1022E40077657273206F6E2069742E2054686520A0
:1022F400666C6F776572732061726520626C6F6FB4
:102304006D696E672E00596F7520656E7465722055
:10231400746865206174746963206F6620746865ED
:1023240020686F7573652E2049742068617320617D
:102334002066657720626F6F6B7320616E64207313
:102344006F6D652066696C657273207769746820A7
:10235400646F63756D656E747320696E736964650B
:102364002069742E205468652066696C6572732038
:1023740061726520676C75656420746F6765746845
:1023840065722E2054686520626F6F6B7320746FC2
:102394006F2E20596F752063616E277420737461EA
:1023A4006E642075702073747261696768742E009E
:1023B400596F7520656E746572207468652062615A
:1023C40073656D656E742E20596F752066696E6431
:1023D40020736F6D6520706F7461746F657320690D
:1023E4006E206120636F726E657220616E6420617D
:1023F40020736B656C65746F6E2061746F702069F7
:10240400742E2000596F7520656E746572206120EA
:10241400726F6F6D207768696368206C6F6F6B7380
:10242400206C696B6520796F7527766520747261FD
:1024340076656C65642066726F6D20616E206F6CCA
:102444006420686F75736520746F207468652063F9
:10245400616D707573206F66206120756E69766595
:1024640072736974792E20546865726520697320CB
:1024740061206C61726765206D616368696E6520B7
:102484007769746861207369676E202044494749FD
:1024940054414C206F6E2069742E204974206C6F57
:1024A4006F6B73206C696B65206120636F6D707551
:1024B4007465722C2074686F75676820796F75274E
:1024C4007665206E65766572207365656E206F6E25
:1024D4006520696E20706572736F6E206265666F29
:1024E40072652E2E2E004E4F5448494E47004C4FD5
:1024F4004E454C5920524F414400532F4E204449DD
:10250400525420524F41440046495245504C414395
:102514004500452F5720537472656574004F4C4431
:1025240020484F555345004C4956494E4720524F79
:102534004F4D00415454494300424153454D454E8B
:102544005400434F4D505554455220524F4F4D0067
:1025540068656C70006E6F72746800736F75746870
:1025640000776573740065617374006465736372E6
:102574006962650075736500696E76656E746F7265
:1025840079007365617263680074616B650045521C
:10259400524F5200496E76616C696420636F6D6DB1
:1025A400616E642100596F752063616E2774207514
:1025B400736520746861742100596F752063616EBE
:1025C400277420676F207468617420776179210013
:1025D400594F55204D415920414354204E4F5721C6
:1025E400005468657265206973206E6F7468696E43
:1025F4006720686572652E2E0069742064696564BD
:10260400006974207375727669766564006120626E
:1026140065617220626C6F636B73207468652077E8
:1026240061790069742072616E20617761792E2E60
:102634002E00697420776F6E27742073746172742E
:1026440000796F752063616E27742074797065005A
:10265400796F7520756E6C6F636B65642074686543
:1026640020646F6F7200576861742061726520790D
:102674006F7520676F696E6720746F20646F3F0009
:10268400596F752074726176656C2061206269747B
:1026940020746F776172647320746865206D6F6F46
:1026A4006E2C20796F75207468696E6B2074686174
:1026B400742773207468652077617920746F2067AC
:1026C4006F2E20596F752066696E642061206265E3
:1026D400617220696E20746865206D6964646C653C
:1026E400206F662074686520726F616420736C6566
:1026F4006570696E67207365656D696E676C7920B6
:10270400696E2070656163652E2054686520776169
:102714007920746F20746865206E6F727468206904
:102724007320626C6F636B656420627920746865E2
:1027340020626561722E00596F7520617472617632
:10274400656C20612062697420746F7761726473B0
:1027540020746865206D6F6F6E2C20796F75204B27
:102764004E4F57207468617427732074686520770E
:10277400617920746F20676F2E20596F7520736DF7
:10278400656C6C20736F6D657468696E672077651E
:102794006972656420616C6F6E6720746865207768
:1027A40061792C2062757420796F7520646F6E27AF
:1027B40074206B6E6F77207768657265206974206A
:1027C400697320636F6D696E672066726F6D2E206A
:1027D400536D656C6C73206C696B6520666C6573F6
:1027E4006820726F7474696E6720617761792E2E28
:0227F4002E00B5
:00000001FF
